:020000040000FA
:020000001628C0
:08000800C92C82073F340634C5
:100010005B344F3466346D347D3407347F346F3451
:1000200000340234043408341034203403138312AF
:100030008501860187019F018316031788018901C5
:10004000031375308F007030850001308600870102
:1000500008308900C33081000C10831200308B00FF
:10006000013090008601861700003230051B3C30BD
:10007000A100A3000310A30CA30C0B160B178B17E6
:100080008030A20086018614221C871422180714CF
:10009000B7248701860106170000051F4228860144
:1000A000A2012108A3001230A500A601A70101307A
:1000B000A400AC00AE01B101B001B401B201B601BF
:1000C000B701C0018316A73084003C30A400800132
:1000D000840AA40B67288312341706308100FA3093
:1000E000A0008B1631187F28AD01AB012408BC227B
:1000F0002508A9002608AA00B71BB71D0D23C0308C
:10010000B405023086002B088700B724FE2000309B
:100110008700043086002A080F390520B71F92286F
:10012000371A80388700B724FE2000308700083057
:1001300086002A0E0F390520B71FA028371A8038ED
:100140008700B724FE200030870010308600290881
:100150000F3905208700B724FE20003087002030AB
:100160008600290E0F39031DB828B71BB71D0A30AA
:1001700005208700B724FE2000308700403086002D
:100180002C088700B724FE200030870080308600CE
:100190002D088700B724FE20003087008601340830
:1001A000C0390319E628341BD7282B21E628B41BB5
:1001B000E62834081F39153C031DE6282008031DD6
:1001C000E628063081004B30A0008B163018D22371
:1001D0008B1AFD2840080319FD28401CF1289124A2
:1001E000FC28C01CF528A524FC28401DF9287224F1
:1001F000FC28C01DFC287924C0017228B41B2A29C0
:100200000508F039B3008919B713891DB717331AD8
:1002100022290730B407B31A22290730B407331B49
:100220001B291F303405143C031919290D30B40261
:100230002A29B40A2A291F303405143C031D222917
:10024000B71F1929341B2A29B41706308100193029
:10025000A0008B16080034081F39B5003618332962
:10026000311837293114E322AF01B801B6010A3041
:10027000350203186829AF1F4429E322AF13311D4B
:100280004429310E0339AB000430B9000310AA0D24
:10029000A90DB90B46293508AA042908F039031914
:1002A0005529A03C031D67295729A030A904290816
:1002B0000F3903195F290A3C031D672961290A3098
:1002C000A9042A08F039031D6729A030AA04A32A2B
:1002D0000C30350203187829AF1BE322AB01351C23
:1002E000AB1435182B140F30B1052B0EB104A32A13
:1002F0000E3035020318C5293808031DAE292A0817
:100300000F39BA000A3C0319B52935189429083069
:100310003A020318C4293A08BC22E330AF05BA0DEB
:100320003A0D1C39AF04AB29AC0105303A02031C6D
:10033000A329B71FC42909303A02031DC429B716DF
:100340000F30AD00AA293A08CC22E030AF053A08B8
:100350000339AF04B114B817E622C429B81EB32973
:100360008030B805B829381BB8296D233817C4293F
:10037000E322351CB722351CC329B71EC2290F3012
:10038000AD00C329CA223813A32A1130350203183D
:100390002F2AB11C9C2AB71ED0293518F9299C2A6E
:1003A000351ADB29351CAB1635182B179F30AF05D6
:1003B000351CAF16DE29AB176030AF042B080339AC
:1003C0000319EA292C08031D1F2A311D9C2ACA2261
:1003D000B7221F2A2C08031D9C2A2A080F390A3C21
:1003E0000319F429CA22122A2D0803199C2A351A46
:1003F000012A2D08351C8504FF3A35188505311072
:100400002E2A0130A900AA013B23AF12A917B3235A
:1004100003189A2AA9130D23B722AB132B172D0803
:1004200085042E2A3214EA2203189C2A3B23A9179A
:10043000B32303189A2AA9130D23B7222E2A3210A8
:10044000EA2203189C2A0319F4292908BA00282350
:10045000B32303189A2A3A08A9003115A32A031DC9
:10046000362AB1103111AF01E322A32A133035022D
:100470000318762AB71E3E2AB712742A0330AD0835
:10048000031D462A1C30AC0803195E2A8316A600F9
:1004900083122F088316A000A73084001430A40014
:1004A000801F582A2008260500062605031980010A
:1004B00003308407A40B502A8312742AB71F682ABA
:1004C000B70A37080739053C031D752AF830B70508
:1004D0008316A73084003C30A4008001840AA40B5A
:1004E0006D2A8312B71F8501B101932A031D962A35
:1004F000AF1B932A2C080319932A2B0803390319DD
:10050000932AB201EA2203189C2A0319932AAF0CFA
:100510002F0C073903190130A40028232908A5004E
:100520002A08A600A701AC01B101A32A0830B7062A
:100530003110A32A88309D2A9930AA00A900AB0166
:10054000AC01AD0136140C3035020319B02A0D3060
:1005500035020319B02AB801B71EB02AB712AD018F
:1005600012303502F830031DB705341708002F0884
:10057000B900B90C390C07390319C72AB900013081
:10058000AC00B9030319C92A0310AC0DC12A7F308E
:10059000AC0008002F08033903190430B9000130FA
:1005A000AD00B9030319D72A0310AD0DD12A0800F5
:1005B0000330AB054030AF1EE12A20302F1FE12A67
:1005C0008030AB040800AB01AC01AD01AA30AA0039
:1005D000A90008002908F039A03C031DF92A0F30B2
:1005E000A90529080A3C031DF92A123032180030E7
:1005F000A900133032181230290203180C2B2A08D4
:10060000F039A03C031D0A2B0F30AA052A080A3C2A
:1006100003190C2B60302A0208002908031D132B34
:100620001230A900172B123029020318192BAB1412
:10063000272B0319262BA9000E302902031C262B79
:10064000103029020318262B0630A9022B140800AB
:100650002908123C0319A9012B1C3A2B1230A907B7
:100660001A302902031C3A2B2230290203183A2B94
:100670000630A9070800E330AF052408BA00BA0D18
:100680003A0D1C39AF042608AA072A080F39093C7D
:100690000630031CAA072A08593C0318522B603065
:1006A000AA02A90A2508A90729080F39093C06301A
:1006B000031CA9072908233C03186C2B2430A9022A
:1006C0002F081C39043E1C390319692B0430A0077C
:1006D0006C2BE330AF052F1508002F088316A00000
:1006E000831238081F398316A50083120030B71A09
:1006F000803035048316A600A73084001430A4008F
:10070000801F942BA61B902B200826188B2B1C399E
:1007100000061C398E2B033900060339031D942B68
:10072000250803199C2BA50303308407A40B802BF9
:100730008312B816E322B22B00088312AF0083168F
:10074000840A000883127F39A9008316840A0008EE
:100750008312AA00B80AAB01B71BB71D0D23B7223D
:10076000CA22D82208008316A73084001430A400BF
:10077000801FC02B03308407A40BB82B0314D02B8D
:100780008312AF172F0883168000840A831229086A
:1007900083168000840A83122A08831680000310BF
:1007A0008312080024088316A100831225088316EB
:1007B000A200831226088316A3000310A10DA10D29
:1007C000A73084001430A400801F572C00081C3967
:1007D0000319ED2B2106031D572C0008A000840AE5
:1007E00000087F392202031D582C840A00082302C6
:1007F000031D592C20088312BA000339B9000319CC
:1008000039150130AE00B9030319092C0310AE0DE0
:10081000032C2E08BA1A8504FF3ABA1E8505B71FA5
:10082000152CBA1A4014BA1EC01483168403801FF4
:10083000202C201F1D2CA01A222C84038001572C51
:10084000201F582C840320308006840AA01A3A2CDA
:100850006824F9300002031D582C233080001C301E
:10086000A0050319582C0430A002031D522C1C3083
:10087000A000522C0008A60080135F242430000240
:1008800003188001A61B80177F300005031D582C1C
:100890001C30A0050319582C0430A007A01E522CB0
:1008A0000430A0008403E3308005A0008004840AA3
:1008B000840A840AA40BE42B831230100800800AF7
:1008C00000080F390A3C031D0800063080070800A5
:1008D00000080F3903196E2C8003080080030630CE
:1008E00080020800F730BE001F30BF006430A9242A
:1008F00008007C247C247C24FB30BE009030BF00A8
:10090000FA30A9240800F630BE000930BF00643078
:10091000A9240800F830BE008930BF006430A92443
:1009200008009324BF248324BF248A240800F130C4
:10093000BE001230BF006430A9240800F130BE00B0
:100940001230BF00FA30A92408009724C1249E2445
:10095000080083160C148312C42483160C1083120F
:1009600008002730BB00B42CBB0BB32C08000330AD
:10097000BA2C0A30BC00B124BC0BBB2C08001E30C2
:10098000C42C6430C42CFA30BD00B924BD0BC52C76
:100990000800F000030E8301F1000A08F2008A014A
:1009A0008B18D72C0B19F52C0C18012D082D8B103A
:1009B000A3030319E52CA21B082DB71F082D031054
:1009C000210C23020319F22C082D2108A300A21FD9
:1009D000EF2C0310A30CA30C0130A206082D0F2549
:1009E000B71F082D1030B706082D0B1106308100F7
:1009F000A00B082D8B12B41FFF2CB413082D341339
:100A0000082D0C103E088F003F088E0080308506B0
:100A100072088A00710E8300F00E700E09002730F4
:100A200084005F2460302702031C372DA701301497
:100A3000263084005F2460302602031C372DA60177
:100A4000B71BC015253084005F2424302502031C09
:100A5000372DA501A40A08302402031C312D0130D2
:100A6000A4003118372D0310AC0D0318AC0DB71FBF
:100A7000412D59302602031D412D573027020318FE
:040A80004015080015
:02400E00C423C9
:02401000FF3F70
:1042000043006F0070007900720069006700680069
:1042100074002000280043002900200032003000F4
:104220003100390020006200790020004D002E008E
:10423000590061006D0061006D006F0074006F0037
:00000001FF
